:020000040000FA
:020000000D28C9
:080008008C0003088D008F0A33
:100010000B110D0883000C080900831605308100C0
:10002000063085000030860083128501860181013B
:100030000B118B168B173F2086158E0105191C2876
:100040008E0A462005300E02031D1E28851C372807
:1000500006163F203F2006128E013C300E02031987
:10006000372846208E0A05191C2885182D280519C1
:100070001C2886114620051D3A2886151C288F014C
:1000800081011F300F02031D412808008F018101EB
:0A00900099300F02031D48280800F4
:02400E00F23F7F
:00000001FF
